:02000000C9280D
:10000800E628A601A500BA172730A400103018204A
:100018000330A400E8301820A40164301820A4019B
:100028000A30182025082328A3002608A20025083E
:10003800A100A8202108031DBA13BA1B0800303EEE
:10004800A7003E0884000930A80003103020A70C40
:10005800A80B2A28031430288413BA1D3F28000847
:100068003C043A1D3C068000841700083C04031C2D
:100078003C0680004A2800083C04031C3C063A1948
:100088003C06800084173C0980054A283A0D063949
:10009800A1005320A200A10A532000006D280030BF
:1000A8008A00210882070134993403343934003432
:1000B80060340C34FD34A401A300FF30A307031CF3
:1000C800A407031CC4280330A200E6306D20612871
:1000D800A201FC3EA100A209031C7828FF30000001
:1000E800A10703187328A1076400A20F722808004B
:1000F800A201A401A30002308D28A201A401A3003B
:1001080001308D28A30004308D28A201A401A3008A
:100118000530A90024082202031D9428230821027F
:10012800043003180130031902302905031DFF307C
:10013800C4280038031DFF300405031DFF30C42800
:100148000404031DFF30C428A601A5011030A70030
:10015800220DA50DA60D2308A5022408031C240FB3
:10016800A6020318BE282308A50724080318240F8D
:10017800A6070310A10DA20DA70BAC282108C428BF
:100188008313031383126400080048108316811335
:100198000C3086008501831207309F0031309000B3
:1001A800C0308B00831601308C008312DC30C30012
:1001B8000B30C2000C30C600C701CA01C101C4011E
:1001C800C5014129A000030E8301C0000A08BB0035
:1001D80043088E0042088F00C10A0C103B088A00B1
:1001E800400E8300A00E200E090064000A30410270
:1001F800031C402983168C0183124108A100A20127
:100208000A30A300A401A820B3002208B4003308D0
:10021800CA074108A100A2010A30A300A401A8202E
:10022800B3002208B4003308C40734080318013E99
:10023800C5074108A100A2010A30A300A401A82013
:100248002508C100831601308C0064003C308312FD
:100258004A02031C40293C30CA02C70A64003C30E9
:100268004702031C4029C701C60A64000D30460234
:10027800031C40290130C60008003322F920440835
:10028800A1004508A200A40109308620031D6C299D
:100298000930C4020030031C013EC5020030861933
:1002A8000130A10000308920B30000300619013068
:1002B800A10000308920B5003308840035089D204E
:1002C800B500B60064003508360403196C29F1221C
:1002D8004908A1004A088920B30000308619013076
:1002E800A10000308920B5003308840035089D201E
:1002F800B500B600003006190130A1000030892091
:10030800B70035083604840037089D20B700B800C8
:1003180064003708380403199429A4234A08C9003B
:10032800003086190130A10000307C20B300003075
:1003380006190130A10000307C20B5003308840084
:1003480035089D20B500B600640035083604031949
:10035800BD29061283160612831286128316861288
:1003680083120613831606138312861383168613C5
:100378008312003086190130A10000307C20B300C0
:10038800003006190130A10000308920B50033087B
:10039800840035089D20B500B60064003508360491
:1003A8000319EF2929230930CA0764003C304A029F
:1003B800031CEF293C30CA02C70A64003C304702DC
:1003C800031CEF29C701C60A64000D304602031C4E
:1003D800EF290130C600003006190130A1000030B5
:1003E8007C20B300003086190130A100003089203C
:1003F800B5003308840035089D20B500B6006400B8
:10040800350836040319322A61230930CA02640008
:1004180065304A02031C322A3C30CA07C70364000D
:1004280065304702031C322A3B30C700C603460822
:10043800A10000307C20B3004608A1006430812070
:10044800B500330884003508A420B500B600640060
:10045800350836040319322A0C30C600422906161C
:1004680083160612831286128316861283120613C7
:100478008316061383128613831686138312992311
:100488000630BE000130BC000630BA0047302420D8
:10049800653024206130242072302420203024202C
:1004A800433024206C3024206F30242063302420F3
:1004B8006B30242020302420493024206E30242022
:1004C80069302420743024206930242061302420AD
:1004D8006C302420693024207A302420693024208C
:1004E8006E3024206730242099230630BE00013066
:1004F800BC000630BA00283024206330242029307C
:100508002420203024203230242030302420303061
:1005180024203930242020302420413024206C30FD
:1005280024207430242061302420203024205430AA
:100538002420653024206330242068302420203093
:100548002420493024206E30242064302420753043
:100558002420733024207430242072302420693001
:100568002420653024207330242099230630BE00CF
:100578000130BC000630BA00443024206530242005
:100588007330242069302420673024206E302420E2
:100598006530242064302420203024206230242038
:1005A8007930242020302420413024206C3024202D
:1005B800613024206E302420203024205030242024
:1005C8006130242072302420653024206B302420B0
:1005D80068302420992399230800861783168613E8
:1005E8001E3083125F200612831606121E308312F5
:1005F8005F200617831606131E3083125F208613AA
:10060800831686131E3083125F2086168316861281
:100618001E3083125F200613831606131E308312C2
:100628005F200616831606121E3083125F2086127C
:10063800831686121E3083125F206400481C282B04
:10064800061283160612831208008617831686136D
:100658000A3083125F200612831606120A308312AC
:100668005F200617831606130A3083125F2086134D
:10067800831686130A3083125F2086168316861225
:100688000A3083125F200613831606130A3083127A
:100698005F200616831606120A3083125F20861220
:1006A800831686120A3083125F206400481C602B70
:1006B80006128316061283120800861683168612FF
:1006C8000A3083125F200612831606120A3083123C
:1006D8005F200617831606130A3083125F208612DE
:1006E800831686120A3083125F20861783168613B4
:1006F8000A3083125F200613831606130A3083120A
:100708005F200616831606120A3083125F208613AE
:10071800831686130A3083125F206400481C982BC6
:10072800061283160612831208000630BE00013036
:10073800BC000630BA000A3024200D3024200800FE
:100748000630BE000130BC000630BA004330242019
:100758007530242072302420723024206530242003
:100768006E3024207430242020302420743024203B
:10077800693024206D302420653024202030242046
:100788006930242073302420203024204608052096
:100798003A302420470805202E3024204A08052016
:1007A8002D302420410805200630BE000130BC0051
:0E07B8000630BA000A3024200D30242008003C
:02400E00463F2B
:00000001FF
